BL51 BANKED LINKER/LOCATER V6.22                                                        01/21/2022  11:42:17  PAGE 1


BL51 BANKED LINKER/LOCATER V6.22, INVOKED BY:
D:\KEIL_V5\C51\BIN\BL51.EXE STARTUP.obj, main.obj, LCD.obj, sys.obj, font.obj, touch.obj TO ceshi RAMSIZE (256)


MEMORY MODEL: LARGE WITH FLOATING POINT ARITHMETIC


INPUT MODULES INCLUDED:
  STARTUP.obj (?C_STARTUP)
  main.obj (MAIN)
  LCD.obj (LCD)
  sys.obj (SYS)
  font.obj (FONT)
  touch.obj (TOUCH)
  D:\KEIL_V5\C51\LIB\C51FPL.LIB (?C?FPADD)
  D:\KEIL_V5\C51\LIB\C51FPL.LIB (?C?FPMUL)
  D:\KEIL_V5\C51\LIB\C51FPL.LIB (?C?FPDIV)
  D:\KEIL_V5\C51\LIB\C51FPL.LIB (?C?FPCMP)
  D:\KEIL_V5\C51\LIB\C51FPL.LIB (?C?FCAST)
  D:\KEIL_V5\C51\LIB\C51FPL.LIB (?C?CASTF)
  D:\KEIL_V5\C51\LIB\C51FPL.LIB (?C?FPGETOPN)
  D:\KEIL_V5\C51\LIB\C51L.LIB (?C_INIT)
  D:\KEIL_V5\C51\LIB\C51L.LIB (?C?CLDPTR)
  D:\KEIL_V5\C51\LIB\C51L.LIB (?C?IMUL)
  D:\KEIL_V5\C51\LIB\C51L.LIB (?C?UIDIV)
  D:\KEIL_V5\C51\LIB\C51L.LIB (?C?IILDX)
  D:\KEIL_V5\C51\LIB\C51L.LIB (?C?ISTPTR)
  D:\KEIL_V5\C51\LIB\C51L.LIB (?C?LMUL)
  D:\KEIL_V5\C51\LIB\C51L.LIB (?C?ULDIV)
  D:\KEIL_V5\C51\LIB\C51L.LIB (?C?LNEG)
  D:\KEIL_V5\C51\LIB\C51L.LIB (?C?ULCMP)
  D:\KEIL_V5\C51\LIB\C51L.LIB (?C?LSTXDATA)
  D:\KEIL_V5\C51\LIB\C51L.LIB (?C?LSTKXDATA)


LINK MAP OF MODULE:  ceshi (?C_STARTUP)


            TYPE    BASE      LENGTH    RELOCATION   SEGMENT NAME
            -----------------------------------------------------

            * * * * * * *   D A T A   M E M O R Y   * * * * * * *
            REG     0000H     0008H     ABSOLUTE     "REG BANK 0"
            IDATA   0008H     0001H     UNIT         ?STACK

            * * * * * * *  X D A T A   M E M O R Y  * * * * * * *
            XDATA   0000H     0082H     UNIT         _XDATA_GROUP_
            XDATA   0082H     0016H     UNIT         ?XD?LCD
            XDATA   0098H     0010H     UNIT         ?XD?TOUCH
            XDATA   00A8H     0001H     UNIT         ?XD?MAIN

            * * * * * * *   C O D E   M E M O R Y   * * * * * * *
            CODE    0000H     0003H     ABSOLUTE     
            CODE    0003H     1370H     UNIT         ?CO?FONT
            CODE    1373H     0CA1H     UNIT         ?PR?TOUCH_ADJUST?TOUCH
            CODE    2014H     0604H     UNIT         ?C?LIB_CODE
            CODE    2618H     01F7H     UNIT         ?PR?_DRAW_CIRCLE?LCD
            CODE    280FH     01F2H     UNIT         ?PR?XIANSHI?MAIN
BL51 BANKED LINKER/LOCATER V6.22                                                      01/21/2022  11:42:17  PAGE 2


            CODE    2A01H     01EBH     UNIT         ?PR?_LCD_DRAWLINE?LCD
            CODE    2BECH     01A5H     UNIT         ?PR?LCD_INIT?LCD
            CODE    2D91H     019EH     UNIT         ?PR?_LCD_SHOWCHAR?LCD
            CODE    2F2FH     0157H     UNIT         ?PR?_ADS_READ_XY?TOUCH
            CODE    3086H     0131H     UNIT         ?PR?_READ_ADS2?TOUCH
            CODE    31B7H     0115H     UNIT         ?PR?SHOWIMAGE?MAIN
            CODE    32CCH     0103H     UNIT         ?PR?CONVERT_POS?TOUCH
            CODE    33CFH     00E8H     UNIT         ?PR?_DROW_TOUCH_POINT?TOUCH
            CODE    34B7H     00E1H     UNIT         ?PR?_LCD_SHOWNUM?LCD
            CODE    3598H     00D9H     UNIT         ?PR?POINT?TOUCH
            CODE    3671H     00CFH     UNIT         ?PR?_SHOWHANZI?LCD
            CODE    3740H     00AAH     UNIT         ?PR?_LCD_DRAWRECTANGLE?LCD
            CODE    37EAH     00A1H     UNIT         ?PR?_LCD_SHOWSTRING?LCD
            CODE    388BH     008CH     UNIT         ?C_C51STARTUP
            CODE    3917H     0086H     UNIT         ?PR?_LCD_FILL?LCD
            CODE    399DH     0082H     UNIT         ?PR?_LCD_SHOW2NUM?LCD
            CODE    3A1FH     007BH     UNIT         ?PR?READ_TP_ONCE?TOUCH
            CODE    3A9AH     006BH     UNIT         ?CO?TOUCH
            CODE    3B05H     0063H     UNIT         ?PR?_READ_ADS?TOUCH
            CODE    3B68H     005EH     UNIT         ?PR?JIANCE?MAIN
            CODE    3BC6H     005CH     UNIT         ?PR?_LCD_CLEAR?LCD
            CODE    3C22H     0052H     UNIT         ?PR?_LCD_DRAWPOINT?LCD
            CODE    3C74H     004CH     UNIT         ?PR?_LCD_DRAWPOINT_BIG?LCD
            CODE    3CC0H     0049H     UNIT         ?C_INITSEG
            CODE    3D09H     0049H     UNIT         ?PR?_MYPOW?LCD
            CODE    3D52H     003AH     UNIT         ?PR?_ADDRESS_SET?LCD
            CODE    3D8CH     0033H     UNIT         ?PR?MAIN?MAIN
            CODE    3DBFH     0029H     UNIT         ?CO?MAIN
            CODE    3DE8H     0026H     UNIT         ?PR?_DELAYMS?SYS
            CODE    3E0EH     0022H     UNIT         ?PR?READFROMCHARFROM7843?TOUCH
            CODE    3E30H     001AH     UNIT         ?PR?_WRITECHARTO7843?TOUCH
            CODE    3E4AH     0017H     UNIT         ?PR?_ADS_READ_AD?TOUCH
            CODE    3E61H     0014H     UNIT         ?PR?_LCD_WR_DATA?LCD
            CODE    3E75H     000EH     UNIT         ?PR?_LCD_WR_REG_DATA?LCD
            CODE    3E83H     000BH     UNIT         ?PR?_LCD_WRIT_BUS?LCD
            CODE    3E8EH     000BH     UNIT         ?PR?_LCD_WR_REG?LCD
            CODE    3E99H     0009H     UNIT         ?PR?SPISTAR?TOUCH
            CODE    3EA2H     0006H     UNIT         ?PR?TPSTATE?TOUCH
            CODE    3EA8H     0005H     UNIT         ?PR?_LCD_WR_DATA8?LCD
            CODE    3EADH     0002H     UNIT         ?CO?LCD



OVERLAY MAP OF MODULE:   ceshi (?C_STARTUP)


SEGMENT                                  XDATA_GROUP
  +--> CALLED SEGMENT                  START    LENGTH
------------------------------------------------------
?C_C51STARTUP                          -----    -----
  +--> ?PR?MAIN?MAIN
  +--> ?C_INITSEG

?PR?MAIN?MAIN                          -----    -----
  +--> ?PR?SPISTAR?TOUCH
  +--> ?PR?LCD_INIT?LCD
  +--> ?PR?_LCD_CLEAR?LCD
BL51 BANKED LINKER/LOCATER V6.22                                                      01/21/2022  11:42:17  PAGE 3


  +--> ?PR?SHOWIMAGE?MAIN
  +--> ?PR?JIANCE?MAIN

?PR?LCD_INIT?LCD                       -----    -----
  +--> ?PR?_LCD_WR_REG_DATA?LCD
  +--> ?CO?LCD
  +--> ?PR?_LCD_SHOWSTRING?LCD
  +--> ?PR?_LCD_SHOWNUM?LCD
  +--> ?PR?_LCD_SHOW2NUM?LCD
  +--> ?PR?_LCD_DRAWPOINT_BIG?LCD
  +--> ?PR?_LCD_DRAWRECTANGLE?LCD
  +--> ?PR?_DRAW_CIRCLE?LCD
  +--> ?PR?_DELAYMS?SYS
  +--> ?PR?_LCD_WR_REG?LCD
  +--> ?PR?_LCD_WR_DATA?LCD

?PR?_LCD_WR_REG_DATA?LCD               -----    -----
  +--> ?PR?_LCD_WR_REG?LCD
  +--> ?PR?_LCD_WR_DATA?LCD

?PR?_LCD_WR_REG?LCD                    -----    -----
  +--> ?PR?_LCD_WRIT_BUS?LCD

?PR?_LCD_WR_DATA?LCD                   -----    -----
  +--> ?PR?_LCD_WRIT_BUS?LCD

?PR?_LCD_SHOWSTRING?LCD                0043H    0007H
  +--> ?PR?_LCD_CLEAR?LCD
  +--> ?PR?_LCD_SHOWCHAR?LCD

?PR?_LCD_CLEAR?LCD                     004AH    0003H
  +--> ?PR?_ADDRESS_SET?LCD
  +--> ?PR?_LCD_WR_DATA8?LCD

?PR?_ADDRESS_SET?LCD                   0063H    0008H
  +--> ?PR?_LCD_WR_REG?LCD
  +--> ?PR?_LCD_WR_DATA?LCD

?PR?_LCD_WR_DATA8?LCD                  -----    -----
  +--> ?PR?_LCD_WRIT_BUS?LCD

?PR?_LCD_SHOWCHAR?LCD                  004FH    000CH
  +--> ?PR?_ADDRESS_SET?LCD
  +--> ?CO?FONT
  +--> ?PR?_LCD_WR_DATA?LCD
  +--> ?PR?_LCD_DRAWPOINT?LCD

?PR?_LCD_DRAWPOINT?LCD                 -----    -----
  +--> ?PR?_ADDRESS_SET?LCD
  +--> ?PR?_LCD_WR_DATA?LCD

?PR?_LCD_SHOWNUM?LCD                   0043H    000CH
  +--> ?PR?_MYPOW?LCD
  +--> ?PR?_LCD_SHOWCHAR?LCD

?PR?_MYPOW?LCD                         004FH    0006H

BL51 BANKED LINKER/LOCATER V6.22                                                      01/21/2022  11:42:17  PAGE 4


?PR?_LCD_SHOW2NUM?LCD                  0000H    0009H
  +--> ?PR?_MYPOW?LCD
  +--> ?PR?_LCD_SHOWCHAR?LCD

?PR?_LCD_DRAWPOINT_BIG?LCD             -----    -----
  +--> ?PR?_LCD_FILL?LCD

?PR?_LCD_FILL?LCD                      000AH    000CH
  +--> ?PR?_ADDRESS_SET?LCD
  +--> ?PR?_LCD_WR_DATA?LCD

?PR?_LCD_DRAWRECTANGLE?LCD             0000H    0008H
  +--> ?PR?_LCD_DRAWLINE?LCD

?PR?_LCD_DRAWLINE?LCD                  0047H    001CH
  +--> ?PR?_LCD_DRAWPOINT?LCD

?PR?_DRAW_CIRCLE?LCD                   0000H    000AH
  +--> ?PR?_LCD_DRAWPOINT?LCD

?PR?SHOWIMAGE?MAIN                     0000H    0006H
  +--> ?PR?_LCD_CLEAR?LCD
  +--> ?PR?XIANSHI?MAIN
  +--> ?PR?_ADDRESS_SET?LCD
  +--> ?PR?JIANCE?MAIN
  +--> ?CO?FONT
  +--> ?PR?_LCD_WR_DATA8?LCD

?PR?XIANSHI?MAIN                       0006H    0004H
  +--> ?PR?_SHOWHANZI?LCD
  +--> ?CO?MAIN
  +--> ?PR?_LCD_SHOWSTRING?LCD
  +--> ?PR?_LCD_SHOWNUM?LCD

?PR?_SHOWHANZI?LCD                     000AH    000AH
  +--> ?CO?FONT
  +--> ?PR?_ADDRESS_SET?LCD
  +--> ?PR?_LCD_WR_DATA?LCD

?PR?JIANCE?MAIN                        -----    -----
  +--> ?PR?TPSTATE?TOUCH
  +--> ?PR?_LCD_CLEAR?LCD
  +--> ?PR?POINT?TOUCH
  +--> ?PR?TOUCH_ADJUST?TOUCH
  +--> ?PR?_DELAYMS?SYS

?PR?POINT?TOUCH                        0006H    0004H
  +--> ?PR?CONVERT_POS?TOUCH
  +--> ?CO?TOUCH
  +--> ?PR?_LCD_SHOWSTRING?LCD
  +--> ?PR?_LCD_SHOWNUM?LCD
  +--> ?PR?_LCD_DRAWPOINT_BIG?LCD

?PR?CONVERT_POS?TOUCH                  000AH    0001H
  +--> ?PR?_READ_ADS2?TOUCH

?PR?_READ_ADS2?TOUCH                   0048H    000EH
BL51 BANKED LINKER/LOCATER V6.22                                                      01/21/2022  11:42:17  PAGE 5


  +--> ?PR?_READ_ADS?TOUCH

?PR?_READ_ADS?TOUCH                    0056H    0008H
  +--> ?PR?_ADS_READ_XY?TOUCH

?PR?_ADS_READ_XY?TOUCH                 005EH    0024H
  +--> ?PR?_ADS_READ_AD?TOUCH

?PR?_ADS_READ_AD?TOUCH                 -----    -----
  +--> ?PR?_WRITECHARTO7843?TOUCH
  +--> ?PR?READFROMCHARFROM7843?TOUCH

?PR?TOUCH_ADJUST?TOUCH                 0006H    003DH
  +--> ?PR?_LCD_CLEAR?LCD
  +--> ?PR?READ_TP_ONCE?TOUCH
  +--> ?PR?_DROW_TOUCH_POINT?TOUCH
  +--> ?CO?TOUCH
  +--> ?PR?_LCD_SHOWSTRING?LCD
  +--> ?PR?_LCD_SHOWNUM?LCD

?PR?READ_TP_ONCE?TOUCH                 0043H    0005H
  +--> ?PR?_READ_ADS2?TOUCH
  +--> ?PR?_DELAYMS?SYS

?PR?_DROW_TOUCH_POINT?TOUCH            0043H    0004H
  +--> ?PR?_LCD_DRAWLINE?LCD
  +--> ?PR?_LCD_DRAWPOINT?LCD



SYMBOL TABLE OF MODULE:  ceshi (?C_STARTUP)

  VALUE           TYPE          NAME
  ----------------------------------

  -------         MODULE        ?C_STARTUP
  C:388BH         SEGMENT       ?C_C51STARTUP
  I:0008H         SEGMENT       ?STACK
  C:0000H         PUBLIC        ?C_STARTUP
  D:00E0H         SYMBOL        ACC
  D:00F0H         SYMBOL        B
  D:0083H         SYMBOL        DPH
  D:0082H         SYMBOL        DPL
  N:0000H         SYMBOL        IBPSTACK
  N:0100H         SYMBOL        IBPSTACKTOP
  N:0080H         SYMBOL        IDATALEN
  C:388EH         SYMBOL        IDATALOOP
  N:0000H         SYMBOL        PBPSTACK
  N:0100H         SYMBOL        PBPSTACKTOP
  N:0000H         SYMBOL        PDATALEN
  N:0000H         SYMBOL        PDATASTART
  N:0000H         SYMBOL        PPAGE
  N:0000H         SYMBOL        PPAGEENABLE
  D:00A0H         SYMBOL        PPAGE_SFR
  D:0081H         SYMBOL        SP
  C:388BH         SYMBOL        STARTUP1
  N:0000H         SYMBOL        XBPSTACK
BL51 BANKED LINKER/LOCATER V6.22                                                      01/21/2022  11:42:17  PAGE 6


  N:0000H         SYMBOL        XBPSTACKTOP
  N:0000H         SYMBOL        XDATALEN
  N:0000H         SYMBOL        XDATASTART
  C:0000H         LINE#         126
  C:388BH         LINE#         133
  C:388DH         LINE#         134
  C:388EH         LINE#         135
  C:388FH         LINE#         136
  C:3891H         LINE#         185
  C:3894H         LINE#         196
  -------         ENDMOD        ?C_STARTUP

  -------         MODULE        MAIN
  C:0000H         SYMBOL        _ICE_DUMMY_
  D:0090H         PUBLIC        P1
  D:00B0H         PUBLIC        P3
  C:3D8CH         PUBLIC        main
  X:00A8H         PUBLIC        ref
  C:31B7H         PUBLIC        showimage
  C:3B68H         PUBLIC        jiance
  C:280FH         PUBLIC        xianshi
  B:00B0H.2       PUBLIC        key1
  B:00B0H.3       PUBLIC        key2
  -------         PROC          JIANCE
  C:3B68H         LINE#         20
  C:3B68H         LINE#         21
  C:3B68H         LINE#         22
  C:3B6EH         LINE#         23
  C:3B6EH         LINE#         24
  C:3B75H         LINE#         25
  C:3B7DH         LINE#         26
  C:3B86H         LINE#         27
  C:3B89H         LINE#         28
  C:3B8CH         LINE#         29
  C:3B8CH         LINE#         30
  C:3B8FH         LINE#         31
  C:3B8FH         LINE#         32
  C:3B92H         LINE#         33
  C:3B95H         LINE#         34
  C:3B95H         LINE#         35
  C:3B9AH         LINE#         36
  C:3B9AH         LINE#         37
  C:3B9FH         LINE#         38
  C:3BA6H         LINE#         39
  C:3BADH         LINE#         40
  C:3BB4H         LINE#         41
  C:3BBBH         LINE#         42
  C:3BC2H         LINE#         43
  C:3BC5H         LINE#         44
  C:3BC5H         LINE#         45
  C:3BC5H         LINE#         46
  -------         ENDPROC       JIANCE
  -------         PROC          XIANSHI
  -------         DO            
  X:0006H         SYMBOL        lx
  X:0008H         SYMBOL        ly
  -------         ENDDO         
BL51 BANKED LINKER/LOCATER V6.22                                                      01/21/2022  11:42:17  PAGE 7


  C:280FH         LINE#         47
  C:280FH         LINE#         48
  C:280FH         LINE#         50
  C:2817H         LINE#         51
  C:2820H         LINE#         52
  C:2829H         LINE#         53
  C:2834H         LINE#         54
  C:2845H         LINE#         55
  C:2871H         LINE#         56
  C:289DH         LINE#         57
  C:28ADH         LINE#         58
  C:28F5H         LINE#         59
  C:2903H         LINE#         60
  C:294FH         LINE#         61
  C:295FH         LINE#         62
  C:29A7H         LINE#         63
  C:29B5H         LINE#         64
  -------         ENDPROC       XIANSHI
  -------         PROC          SHOWIMAGE
  -------         DO            
  X:0000H         SYMBOL        i
  X:0002H         SYMBOL        j
  X:0004H         SYMBOL        k
  -------         ENDDO         
  C:31B7H         LINE#         66
  C:31B7H         LINE#         67
  C:31B7H         LINE#         69
  C:31BEH         LINE#         70
  C:31C1H         LINE#         71
  C:31CAH         LINE#         72
  C:31CAH         LINE#         73
  C:31D1H         LINE#         74
  C:31D1H         LINE#         75
  C:3225H         LINE#         76
  C:322CH         LINE#         77
  C:322CH         LINE#         78
  C:3232H         LINE#         79
  C:3232H         LINE#         80
  C:3239H         LINE#         82
  C:3239H         LINE#         83
  C:3263H         LINE#         84
  C:3282H         LINE#         85
  C:32A4H         LINE#         86
  C:32C6H         LINE#         87
  C:32CBH         LINE#         88
  -------         ENDPROC       SHOWIMAGE
  -------         PROC          MAIN
  C:3D8CH         LINE#         89
  C:3D8CH         LINE#         90
  C:3D8CH         LINE#         91
  C:3D8FH         LINE#         92
  C:3D92H         LINE#         93
  C:3D99H         LINE#         94
  C:3DA8H         LINE#         95
  C:3DABH         LINE#         97
  C:3DABH         LINE#         98
  C:3DABH         LINE#         99
BL51 BANKED LINKER/LOCATER V6.22                                                      01/21/2022  11:42:17  PAGE 8


  C:3DB1H         LINE#         100
  C:3DB1H         LINE#         101
  C:3DB4H         LINE#         102
  C:3DB4H         LINE#         103
  C:3DBDH         LINE#         105
  -------         ENDPROC       MAIN
  -------         ENDMOD        MAIN

  -------         MODULE        LCD
  C:0000H         SYMBOL        _ICE_DUMMY_
  D:0080H         PUBLIC        P0
  D:0090H         PUBLIC        P1
  D:00A0H         PUBLIC        P2
  D:00B0H         PUBLIC        P3
  C:34B7H         PUBLIC        _LCD_ShowNum
  C:2BECH         PUBLIC        Lcd_Init
  C:3EA8H         PUBLIC        _LCD_WR_DATA8
  C:3E75H         PUBLIC        _LCD_WR_REG_DATA
  X:0082H         PUBLIC        HT
  C:3E8EH         PUBLIC        _LCD_WR_REG
  C:3BC6H         PUBLIC        _LCD_Clear
  X:0084H         PUBLIC        VT
  C:399DH         PUBLIC        _LCD_Show2Num
  C:3917H         PUBLIC        _LCD_Fill
  C:3D09H         PUBLIC        _mypow
  C:2618H         PUBLIC        _Draw_Circle
  B:0090H.0       PUBLIC        LCD_CS
  B:00B0H.7       PUBLIC        LCD_RD
  C:2A01H         PUBLIC        _LCD_DrawLine
  C:3C4AH         PUBLIC        _LCD_DrawPoint
  C:37EAH         PUBLIC        _LCD_ShowString
  C:2D97H         PUBLIC        _LCD_ShowChar
  C:3E6AH         PUBLIC        _LCD_WR_DATA
  B:00B0H.5       PUBLIC        LCD_RS
  X:0086H         PUBLIC        HDP
  B:00B0H.6       PUBLIC        LCD_WR
  C:3740H         PUBLIC        _LCD_DrawRectangle
  C:3671H         PUBLIC        _showhanzi
  C:3C74H         PUBLIC        _LCD_DrawPoint_big
  C:3E83H         PUBLIC        _LCD_Writ_Bus
  X:0088H         PUBLIC        FPS
  X:008AH         PUBLIC        VDP
  X:008CH         PUBLIC        HPS
  X:008EH         PUBLIC        POINT_COLOR
  X:0090H         PUBLIC        HPW
  X:0091H         PUBLIC        LPS
  X:0093H         PUBLIC        BACK_COLOR
  B:0090H.2       PUBLIC        LCD_REST
  C:3D52H         PUBLIC        _Address_set
  X:0095H         PUBLIC        VPS
  X:0097H         PUBLIC        VPW
  -------         PROC          _LCD_WRIT_BUS
  D:0007H         SYMBOL        VH
  D:0005H         SYMBOL        VL
  C:3E83H         LINE#         30
  C:3E83H         LINE#         31
  C:3E83H         LINE#         32
BL51 BANKED LINKER/LOCATER V6.22                                                      01/21/2022  11:42:17  PAGE 9


  C:3E85H         LINE#         33
  C:3E89H         LINE#         34
  C:3E8BH         LINE#         35
  C:3E8DH         LINE#         36
  -------         ENDPROC       _LCD_WRIT_BUS
  -------         PROC          _LCD_WR_DATA8
  D:0007H         SYMBOL        VH
  D:0005H         SYMBOL        VL
  C:3EA8H         LINE#         48
  C:3EA8H         LINE#         49
  C:3EA8H         LINE#         50
  C:3EAAH         LINE#         51
  -------         ENDPROC       _LCD_WR_DATA8
  C:3E61H         SYMBOL        L?0111
  C:3E62H         SYMBOL        L?0112
  -------         PROC          L?0110
  -------         ENDPROC       L?0110
  C:3E61H         SYMBOL        L?0111
  C:3E62H         SYMBOL        L?0112
  -------         PROC          _LCD_WR_DATA
  D:0004H         SYMBOL        da
  C:3E6AH         LINE#         53
  C:3E6EH         LINE#         54
  C:3E6EH         LINE#         55
  C:3E70H         LINE#         56
  -------         ENDPROC       _LCD_WR_DATA
  -------         PROC          _LCD_WR_REG
  D:0004H         SYMBOL        da
  C:3E8EH         LINE#         58
  C:3E92H         LINE#         59
  C:3E92H         LINE#         60
  C:3E94H         LINE#         61
  -------         ENDPROC       _LCD_WR_REG
  -------         PROC          _LCD_WR_REG_DATA
  D:0006H         SYMBOL        reg
  D:0002H         SYMBOL        da
  C:3E75H         LINE#         63
  C:3E79H         LINE#         64
  C:3E79H         LINE#         65
  C:3E7CH         LINE#         66
  -------         ENDPROC       _LCD_WR_REG_DATA
  -------         PROC          _ADDRESS_SET
  X:0063H         SYMBOL        x1
  X:0065H         SYMBOL        y1
  D:0002H         SYMBOL        x2
  X:0069H         SYMBOL        y2
  C:3D52H         LINE#         68
  C:3D60H         LINE#         69
  C:3D60H         LINE#         70
  C:3D67H         LINE#         71
  C:3D6AH         LINE#         72
  C:3D6DH         LINE#         73
  C:3D72H         LINE#         74
  C:3D79H         LINE#         75
  C:3D7EH         LINE#         76
  C:3D7EH         LINE#         77
  C:3D81H         LINE#         78
BL51 BANKED LINKER/LOCATER V6.22                                                      01/21/2022  11:42:17  PAGE 10


  C:3D84H         LINE#         79
  C:3D87H         LINE#         80
  -------         ENDPROC       _ADDRESS_SET
  -------         PROC          LCD_INIT
  C:2BECH         LINE#         82
  C:2BECH         LINE#         83
  C:2BECH         LINE#         86
  C:2BEEH         LINE#         87
  C:2BF1H         LINE#         88
  C:2BF1H         LINE#         89
  C:2BF9H         LINE#         90
  C:2C07H         LINE#         91
  C:2C1DH         LINE#         92
  C:2C2BH         LINE#         93
  C:2C33H         LINE#         94
  C:2C43H         LINE#         95
  C:2C4CH         LINE#         96
  C:2C4CH         LINE#         98
  C:2C4EH         LINE#         99
  C:2C55H         LINE#         100
  C:2C57H         LINE#         101
  C:2C5EH         LINE#         102
  C:2C60H         LINE#         103
  C:2C62H         LINE#         104
  C:2C64H         LINE#         105
  C:2C66H         LINE#         106
  C:2C6DH         LINE#         107
  C:2C6FH         LINE#         109
  C:2C76H         LINE#         110
  C:2C7BH         LINE#         111
  C:2C80H         LINE#         112
  C:2C85H         LINE#         113
  C:2C8AH         LINE#         114
  C:2C8FH         LINE#         115
  C:2C94H         LINE#         116
  C:2C9BH         LINE#         117
  C:2CA0H         LINE#         118
  C:2CA5H         LINE#         119
  C:2CACH         LINE#         120
  C:2CB1H         LINE#         121
  C:2CB8H         LINE#         122
  C:2CBDH         LINE#         123
  C:2CC2H         LINE#         124
  C:2CC7H         LINE#         126
  C:2CCCH         LINE#         127
  C:2CD1H         LINE#         128
  C:2CD6H         LINE#         129
  C:2CD9H         LINE#         130
  C:2CDCH         LINE#         131
  C:2CDFH         LINE#         132
  C:2CE2H         LINE#         133
  C:2CE7H         LINE#         134
  C:2CECH         LINE#         135
  C:2CF3H         LINE#         136
  C:2CF6H         LINE#         137
  C:2CF9H         LINE#         138
  C:2CFCH         LINE#         139
BL51 BANKED LINKER/LOCATER V6.22                                                      01/21/2022  11:42:17  PAGE 11


  C:2CFFH         LINE#         140
  C:2D07H         LINE#         141
  C:2D07H         LINE#         142
  C:2D0AH         LINE#         143
  C:2D0FH         LINE#         145
  C:2D14H         LINE#         146
  C:2D17H         LINE#         147
  C:2D1AH         LINE#         148
  C:2D22H         LINE#         149
  C:2D22H         LINE#         150
  C:2D25H         LINE#         151
  C:2D28H         LINE#         152
  C:2D2BH         LINE#         155
  C:2D30H         LINE#         156
  C:2D35H         LINE#         158
  C:2D3AH         LINE#         159
  C:2D3FH         LINE#         162
  C:2D44H         LINE#         165
  C:2D4BH         LINE#         167
  C:2D50H         LINE#         168
  C:2D55H         LINE#         169
  C:2D5AH         LINE#         170
  C:2D5FH         LINE#         171
  C:2D64H         LINE#         172
  C:2D69H         LINE#         173
  C:2D6EH         LINE#         175
  C:2D73H         LINE#         176
  C:2D78H         LINE#         179
  C:2D7DH         LINE#         180
  C:2D82H         LINE#         181
  C:2D87H         LINE#         183
  C:2D8CH         LINE#         184
  -------         ENDPROC       LCD_INIT
  -------         PROC          _LCD_CLEAR
  D:0004H         SYMBOL        Color
  -------         DO            
  X:004AH         SYMBOL        VH
  D:0001H         SYMBOL        VL
  X:004BH         SYMBOL        i
  D:0002H         SYMBOL        j
  -------         ENDDO         
  C:3BC6H         LINE#         188
  C:3BC8H         LINE#         189
  C:3BC8H         LINE#         192
  C:3BCDH         LINE#         193
  C:3BCFH         LINE#         194
  C:3BE5H         LINE#         195
  C:3BECH         LINE#         196
  C:3BECH         LINE#         197
  C:3BEFH         LINE#         198
  C:3BEFH         LINE#         199
  C:3BF9H         LINE#         200
  C:3C04H         LINE#         202
  C:3C21H         LINE#         203
  -------         ENDPROC       _LCD_CLEAR
  -------         PROC          _SHOWHANZI
  X:000AH         SYMBOL        x
BL51 BANKED LINKER/LOCATER V6.22                                                      01/21/2022  11:42:17  PAGE 12


  X:000CH         SYMBOL        y
  X:000EH         SYMBOL        index
  -------         DO            
  X:000FH         SYMBOL        i
  X:0010H         SYMBOL        j
  X:0011H         SYMBOL        temp
  -------         ENDDO         
  C:3671H         LINE#         206
  C:3686H         LINE#         207
  C:3686H         LINE#         209
  C:3694H         LINE#         210
  C:36C0H         LINE#         211
  C:36D3H         LINE#         212
  C:36D8H         LINE#         213
  C:36D8H         LINE#         214
  C:36E7H         LINE#         215
  C:36E7H         LINE#         216
  C:3711H         LINE#         217
  C:3711H         LINE#         218
  C:3714H         LINE#         219
  C:3716H         LINE#         221
  C:3716H         LINE#         222
  C:3721H         LINE#         223
  C:3721H         LINE#         224
  C:3729H         LINE#         225
  C:3733H         LINE#         226
  C:373FH         LINE#         227
  -------         ENDPROC       _SHOWHANZI
  C:3C35H         SYMBOL        L?0114
  C:3C38H         SYMBOL        L?0115
  C:3C39H         SYMBOL        L?0116
  -------         PROC          L?0113
  -------         ENDPROC       L?0113
  C:3C35H         SYMBOL        L?0114
  C:3C38H         SYMBOL        L?0115
  C:3C39H         SYMBOL        L?0116
  -------         PROC          _LCD_DRAWPOINT
  D:0002H         SYMBOL        x
  D:0082H         SYMBOL        y
  C:3C4AH         LINE#         230
  C:3C52H         LINE#         231
  C:3C52H         LINE#         232
  C:3C69H         LINE#         233
  -------         ENDPROC       _LCD_DRAWPOINT
  -------         PROC          _LCD_DRAWPOINT_BIG
  D:0002H         SYMBOL        x
  D:0082H         SYMBOL        y
  C:3C74H         LINE#         237
  C:3C7CH         LINE#         238
  C:3C7CH         LINE#         239
  -------         ENDPROC       _LCD_DRAWPOINT_BIG
  -------         PROC          _LCD_FILL
  X:000AH         SYMBOL        xsta
  X:000CH         SYMBOL        ysta
  X:000EH         SYMBOL        xend
  X:0010H         SYMBOL        yend
  X:0012H         SYMBOL        color
BL51 BANKED LINKER/LOCATER V6.22                                                      01/21/2022  11:42:17  PAGE 13


  -------         DO            
  X:0014H         SYMBOL        i
  D:0002H         SYMBOL        j
  -------         ENDDO         
  C:3917H         LINE#         244
  C:392BH         LINE#         245
  C:392BH         LINE#         247
  C:393FH         LINE#         248
  C:3963H         LINE#         249
  C:3963H         LINE#         250
  C:398CH         LINE#         251
  C:399CH         LINE#         252
  -------         ENDPROC       _LCD_FILL
  -------         PROC          _LCD_DRAWLINE
  X:0047H         SYMBOL        x1
  X:0049H         SYMBOL        y1
  D:0002H         SYMBOL        x2
  X:004DH         SYMBOL        y2
  -------         DO            
  X:004FH         SYMBOL        t
  X:0051H         SYMBOL        xerr
  X:0053H         SYMBOL        yerr
  X:0055H         SYMBOL        delta_x
  X:0057H         SYMBOL        delta_y
  X:0059H         SYMBOL        distance
  X:005BH         SYMBOL        incx
  X:005DH         SYMBOL        incy
  X:005FH         SYMBOL        uRow
  X:0061H         SYMBOL        uCol
  -------         ENDDO         
  C:2A01H         LINE#         256
  C:2A0FH         LINE#         257
  C:2A0FH         LINE#         259
  C:2A1AH         LINE#         262
  C:2A2FH         LINE#         263
  C:2A4AH         LINE#         264
  C:2A59H         LINE#         265
  C:2A5FH         LINE#         266
  C:2A7BH         LINE#         267
  C:2A87H         LINE#         268
  C:2A9CH         LINE#         269
  C:2AB8H         LINE#         270
  C:2AC4H         LINE#         271
  C:2AD9H         LINE#         272
  C:2AFFH         LINE#         273
  C:2B04H         LINE#         274
  C:2B29H         LINE#         275
  C:2B29H         LINE#         276
  C:2B3AH         LINE#         277
  C:2B4EH         LINE#         278
  C:2B62H         LINE#         279
  C:2B7EH         LINE#         280
  C:2B7EH         LINE#         281
  C:2B8AH         LINE#         282
  C:2B9EH         LINE#         283
  C:2B9EH         LINE#         284
  C:2BBAH         LINE#         285
BL51 BANKED LINKER/LOCATER V6.22                                                      01/21/2022  11:42:17  PAGE 14


  C:2BBAH         LINE#         286
  C:2BC6H         LINE#         287
  C:2BDAH         LINE#         288
  C:2BDAH         LINE#         289
  C:2BEBH         LINE#         290
  -------         ENDPROC       _LCD_DRAWLINE
  -------         PROC          _LCD_DRAWRECTANGLE
  X:0000H         SYMBOL        x1
  X:0002H         SYMBOL        y1
  X:0004H         SYMBOL        x2
  X:0006H         SYMBOL        y2
  C:3740H         LINE#         292
  C:3756H         LINE#         293
  C:3756H         LINE#         294
  C:3772H         LINE#         295
  C:3799H         LINE#         296
  C:37C1H         LINE#         297
  -------         ENDPROC       _LCD_DRAWRECTANGLE
  -------         PROC          _DRAW_CIRCLE
  X:0000H         SYMBOL        x0
  X:0002H         SYMBOL        y0
  D:0003H         SYMBOL        r
  -------         DO            
  X:0004H         SYMBOL        a
  X:0006H         SYMBOL        b
  X:0008H         SYMBOL        di
  -------         ENDDO         
  C:2618H         LINE#         302
  C:2626H         LINE#         303
  C:2626H         LINE#         306
  C:2635H         LINE#         307
  C:2649H         LINE#         308
  C:2667H         LINE#         309
  C:2667H         LINE#         310
  C:268CH         LINE#         311
  C:26B8H         LINE#         312
  C:26CFH         LINE#         313
  C:26FCH         LINE#         314
  C:2729H         LINE#         315
  C:2742H         LINE#         316
  C:276EH         LINE#         317
  C:2771H         LINE#         318
  C:278CH         LINE#         319
  C:279AH         LINE#         321
  C:27C9H         LINE#         323
  C:27C9H         LINE#         324
  C:27FAH         LINE#         325
  C:2808H         LINE#         326
  C:2808H         LINE#         327
  C:280BH         LINE#         328
  C:280EH         LINE#         329
  -------         ENDPROC       _DRAW_CIRCLE
  -------         PROC          L?0117
  -------         ENDPROC       L?0117
  -------         PROC          _LCD_SHOWCHAR
  X:004FH         SYMBOL        x
  X:0051H         SYMBOL        y
BL51 BANKED LINKER/LOCATER V6.22                                                      01/21/2022  11:42:17  PAGE 15


  X:0053H         SYMBOL        num
  X:0054H         SYMBOL        mode
  -------         DO            
  X:0055H         SYMBOL        temp
  D:0001H         SYMBOL        pos
  X:0056H         SYMBOL        t
  X:0057H         SYMBOL        x0
  X:0059H         SYMBOL        colortemp
  -------         ENDDO         
  C:2D97H         LINE#         339
  C:2DA8H         LINE#         340
  C:2DA8H         LINE#         343
  C:2DB8H         LINE#         344
  C:2DC7H         LINE#         345
  C:2DE5H         LINE#         347
  C:2DECH         LINE#         348
  C:2E18H         LINE#         349
  C:2E21H         LINE#         350
  C:2E21H         LINE#         351
  C:2E22H         LINE#         352
  C:2E22H         LINE#         353
  C:2E44H         LINE#         354
  C:2E47H         LINE#         355
  C:2E47H         LINE#         356
  C:2E53H         LINE#         357
  C:2E62H         LINE#         358
  C:2E6DH         LINE#         359
  C:2E74H         LINE#         360
  C:2E82H         LINE#         361
  C:2E8EH         LINE#         362
  C:2E9DH         LINE#         363
  C:2EABH         LINE#         364
  C:2EB6H         LINE#         365
  C:2EB6H         LINE#         366
  C:2EB6H         LINE#         367
  C:2EB8H         LINE#         368
  C:2EB8H         LINE#         369
  C:2EDAH         LINE#         370
  C:2EE7H         LINE#         371
  C:2EE7H         LINE#         372
  C:2F0DH         LINE#         373
  C:2F14H         LINE#         374
  C:2F1AH         LINE#         375
  C:2F1FH         LINE#         376
  C:2F1FH         LINE#         377
  C:2F2EH         LINE#         378
  -------         ENDPROC       _LCD_SHOWCHAR
  -------         PROC          _MYPOW
  X:004FH         SYMBOL        m
  X:0050H         SYMBOL        n
  -------         DO            
  X:0051H         SYMBOL        result
  -------         ENDDO         
  C:3D09H         LINE#         380
  C:3D11H         LINE#         381
  C:3D11H         LINE#         382
  C:3D19H         LINE#         383
BL51 BANKED LINKER/LOCATER V6.22                                                      01/21/2022  11:42:17  PAGE 16


  C:3D43H         LINE#         384
  C:3D51H         LINE#         385
  -------         ENDPROC       _MYPOW
  -------         PROC          _LCD_SHOWNUM
  X:0043H         SYMBOL        x
  X:0045H         SYMBOL        y
  X:0047H         SYMBOL        num
  X:004BH         SYMBOL        len
  -------         DO            
  X:004CH         SYMBOL        t
  X:004DH         SYMBOL        temp
  X:004EH         SYMBOL        enshow
  -------         ENDDO         
  C:34B7H         LINE#         391
  C:34C5H         LINE#         392
  C:34C5H         LINE#         394
  C:34CAH         LINE#         395
  C:34DDH         LINE#         396
  C:34F1H         LINE#         397
  C:34F1H         LINE#         398
  C:3522H         LINE#         399
  C:3533H         LINE#         400
  C:3533H         LINE#         401
  C:3537H         LINE#         402
  C:3537H         LINE#         403
  C:3559H         LINE#         404
  C:355BH         LINE#         405
  C:3561H         LINE#         407
  C:3561H         LINE#         408
  C:358EH         LINE#         409
  C:3597H         LINE#         410
  -------         ENDPROC       _LCD_SHOWNUM
  -------         PROC          _LCD_SHOW2NUM
  X:0000H         SYMBOL        x
  X:0002H         SYMBOL        y
  X:0004H         SYMBOL        num
  X:0006H         SYMBOL        len
  -------         DO            
  X:0007H         SYMBOL        t
  X:0008H         SYMBOL        temp
  -------         ENDDO         
  C:399DH         LINE#         414
  C:39B1H         LINE#         415
  C:39B1H         LINE#         417
  C:39C2H         LINE#         418
  C:39C2H         LINE#         419
  C:39F2H         LINE#         420
  C:3A16H         LINE#         421
  C:3A1EH         LINE#         422
  -------         ENDPROC       _LCD_SHOW2NUM
  -------         PROC          _LCD_SHOWSTRING
  X:0043H         SYMBOL        x
  X:0045H         SYMBOL        y
  X:0047H         SYMBOL        p
  C:37EAH         LINE#         427
  C:3801H         LINE#         428
  C:3801H         LINE#         429
BL51 BANKED LINKER/LOCATER V6.22                                                      01/21/2022  11:42:17  PAGE 17


  C:3811H         LINE#         430
  C:3811H         LINE#         431
  C:3832H         LINE#         432
  C:3852H         LINE#         433
  C:386FH         LINE#         434
  C:387DH         LINE#         435
  C:3887H         LINE#         436
  C:388AH         LINE#         437
  -------         ENDPROC       _LCD_SHOWSTRING
  -------         ENDMOD        LCD

  -------         MODULE        SYS
  C:0000H         SYMBOL        _ICE_DUMMY_
  C:3DE8H         PUBLIC        _delayms
  -------         PROC          _DELAYMS
  D:0006H         SYMBOL        count
  -------         DO            
  D:0004H         SYMBOL        i
  D:0002H         SYMBOL        j
  -------         ENDDO         
  C:3DE8H         LINE#         4
  C:3DE8H         LINE#         5
  C:3DE8H         LINE#         7
  C:3DF8H         LINE#         8
  C:3E0DH         LINE#         9
  -------         ENDPROC       _DELAYMS
  -------         ENDMOD        SYS

  -------         MODULE        FONT
  C:0000H         SYMBOL        _ICE_DUMMY_
  C:0003H         PUBLIC        image
  C:0D83H         PUBLIC        asc2_1608
  C:0C83H         PUBLIC        hanzi
  -------         ENDMOD        FONT

  -------         MODULE        TOUCH
  C:0000H         SYMBOL        _ICE_DUMMY_
  D:0090H         PUBLIC        P1
  D:00B0H         PUBLIC        P3
  C:3E0EH         PUBLIC        ReadFromCharFrom7843
  C:3EA2H         PUBLIC        tpstate
  C:3E99H         PUBLIC        spistar
  B:0090H.4       PUBLIC        CS
  B:00D0H.7       PUBLIC        CY
  C:3E4AH         PUBLIC        _ADS_Read_AD
  B:0090H.7       PUBLIC        DCLK
  C:3E30H         PUBLIC        _WriteCharTo7843
  C:3598H         PUBLIC        point
  C:3B05H         PUBLIC        _Read_ADS
  B:00B0H.1       PUBLIC        DOUT
  X:0098H         PUBLIC        chx
  X:009AH         PUBLIC        chy
  C:2F2FH         PUBLIC        _ADS_Read_XY
  X:009CH         PUBLIC        tp_pixlcd
  C:1373H         PUBLIC        Touch_Adjust
  B:00B0H.0       PUBLIC        DIN
  X:00A0H         PUBLIC        tp_pixad
BL51 BANKED LINKER/LOCATER V6.22                                                      01/21/2022  11:42:17  PAGE 18


  C:3086H         PUBLIC        _Read_ADS2
  C:3A1FH         PUBLIC        Read_TP_Once
  X:00A4H         PUBLIC        vx
  X:00A6H         PUBLIC        vy
  C:33CFH         PUBLIC        _Drow_Touch_Point
  B:00B0H.4       PUBLIC        Penirq
  C:32CCH         PUBLIC        Convert_Pos
  -------         PROC          TPSTATE
  C:3EA2H         LINE#         15
  C:3EA2H         LINE#         16
  C:3EA2H         LINE#         17
  C:3EA7H         LINE#         18
  -------         ENDPROC       TPSTATE
  -------         PROC          SPISTAR
  C:3E99H         LINE#         20
  C:3E99H         LINE#         21
  C:3E99H         LINE#         22
  C:3E9BH         LINE#         23
  C:3E9DH         LINE#         24
  C:3E9FH         LINE#         25
  C:3EA1H         LINE#         26
  -------         ENDPROC       SPISTAR
  -------         PROC          _WRITECHARTO7843
  D:0007H         SYMBOL        num
  -------         DO            
  D:0006H         SYMBOL        count
  -------         ENDDO         
  C:3E30H         LINE#         28
  C:3E30H         LINE#         29
  C:3E30H         LINE#         30
  C:3E32H         LINE#         31
  C:3E34H         LINE#         32
  C:3E34H         LINE#         33
  C:3E34H         LINE#         34
  C:3E38H         LINE#         35
  C:3E3AH         LINE#         36
  C:3E3FH         LINE#         37
  C:3E44H         LINE#         38
  C:3E49H         LINE#         39
  -------         ENDPROC       _WRITECHARTO7843
  -------         PROC          READFROMCHARFROM7843
  -------         DO            
  D:0005H         SYMBOL        count
  D:0006H         SYMBOL        Num
  -------         ENDDO         
  C:3E0EH         LINE#         41
  C:3E0EH         LINE#         42
  C:3E0EH         LINE#         43
  C:3E10H         LINE#         44
  C:3E12H         LINE#         45
  C:3E12H         LINE#         46
  C:3E12H         LINE#         47
  C:3E19H         LINE#         48
  C:3E1EH         LINE#         49
  C:3E23H         LINE#         50
  C:3E26H         LINE#         51
  C:3E26H         LINE#         52
BL51 BANKED LINKER/LOCATER V6.22                                                      01/21/2022  11:42:17  PAGE 19


  C:3E2AH         LINE#         53
  C:3E2AH         LINE#         55
  C:3E2FH         LINE#         57
  C:3E2FH         LINE#         58
  -------         ENDPROC       READFROMCHARFROM7843
  -------         PROC          _ADS_READ_AD
  D:0007H         SYMBOL        CMD
  -------         DO            
  D:0006H         SYMBOL        l
  -------         ENDDO         
  C:3E4AH         LINE#         60
  C:3E4AH         LINE#         61
  C:3E4AH         LINE#         63
  C:3E4CH         LINE#         64
  C:3E4FH         LINE#         65
  C:3E55H         LINE#         66
  C:3E5BH         LINE#         67
  C:3E5EH         LINE#         68
  C:3E60H         LINE#         69
  C:3E60H         LINE#         70
  -------         ENDPROC       _ADS_READ_AD
  -------         PROC          _ADS_READ_XY
  D:0001H         SYMBOL        xy
  -------         DO            
  D:0002H         SYMBOL        i
  X:005EH         SYMBOL        j
  X:0060H         SYMBOL        buf
  X:007EH         SYMBOL        sum
  X:0080H         SYMBOL        temp
  -------         ENDDO         
  C:2F2FH         LINE#         76
  C:2F31H         LINE#         77
  C:2F31H         LINE#         80
  C:2F38H         LINE#         82
  C:2F3AH         LINE#         83
  C:2F3AH         LINE#         84
  C:2F59H         LINE#         85
  C:2F64H         LINE#         86
  C:2F67H         LINE#         87
  C:2F67H         LINE#         88
  C:2F87H         LINE#         89
  C:2F87H         LINE#         90
  C:2FB9H         LINE#         91
  C:2FB9H         LINE#         92
  C:2FC1H         LINE#         93
  C:2FF3H         LINE#         94
  C:3017H         LINE#         95
  C:3017H         LINE#         96
  C:302BH         LINE#         97
  C:3039H         LINE#         98
  C:3040H         LINE#         99
  C:3070H         LINE#         100
  C:3085H         LINE#         101
  C:3085H         LINE#         102
  -------         ENDPROC       _ADS_READ_XY
  -------         PROC          _READ_ADS
  X:0056H         SYMBOL        x
BL51 BANKED LINKER/LOCATER V6.22                                                      01/21/2022  11:42:17  PAGE 20


  X:0059H         SYMBOL        y
  -------         DO            
  X:005CH         SYMBOL        xtemp
  D:0006H         SYMBOL        ytemp
  -------         ENDDO         
  C:3B05H         LINE#         105
  C:3B10H         LINE#         106
  C:3B10H         LINE#         108
  C:3B1DH         LINE#         109
  C:3B22H         LINE#         110
  C:3B3CH         LINE#         111
  C:3B54H         LINE#         112
  C:3B65H         LINE#         113
  C:3B67H         LINE#         114
  -------         ENDPROC       _READ_ADS
  -------         PROC          _READ_ADS2
  X:0048H         SYMBOL        x
  X:004BH         SYMBOL        y
  -------         DO            
  X:004EH         SYMBOL        x1
  X:0050H         SYMBOL        y1
  X:0052H         SYMBOL        x2
  X:0054H         SYMBOL        y2
  D:0007H         SYMBOL        flag
  -------         ENDDO         
  C:3086H         LINE#         119
  C:3091H         LINE#         120
  C:3091H         LINE#         124
  C:30A8H         LINE#         125
  C:30ADH         LINE#         126
  C:30C4H         LINE#         127
  C:30C9H         LINE#         128
  C:315FH         LINE#         130
  C:315FH         LINE#         131
  C:3188H         LINE#         132
  C:31B1H         LINE#         133
  C:31B4H         LINE#         134
  C:31B6H         LINE#         135
  -------         ENDPROC       _READ_ADS2
  -------         PROC          READ_TP_ONCE
  -------         DO            
  X:0043H         SYMBOL        re
  X:0044H         SYMBOL        x1
  X:0046H         SYMBOL        y1
  -------         ENDDO         
  C:3A1FH         LINE#         137
  C:3A1FH         LINE#         138
  C:3A1FH         LINE#         139
  C:3A24H         LINE#         141
  C:3A2AH         LINE#         142
  C:3A2AH         LINE#         143
  C:3A44H         LINE#         144
  C:3A4BH         LINE#         145
  C:3A65H         LINE#         146
  C:3A8DH         LINE#         147
  C:3A8DH         LINE#         148
  C:3A92H         LINE#         149
BL51 BANKED LINKER/LOCATER V6.22                                                      01/21/2022  11:42:17  PAGE 21


  C:3A92H         LINE#         150
  C:3A94H         LINE#         151
  C:3A99H         LINE#         152
  -------         ENDPROC       READ_TP_ONCE
  -------         PROC          _DROW_TOUCH_POINT
  X:0043H         SYMBOL        x
  X:0045H         SYMBOL        y
  C:33CFH         LINE#         157
  C:33DDH         LINE#         158
  C:33DDH         LINE#         159
  C:3407H         LINE#         160
  C:343BH         LINE#         161
  C:345AH         LINE#         162
  C:3479H         LINE#         163
  C:3498H         LINE#         164
  -------         ENDPROC       _DROW_TOUCH_POINT
  -------         PROC          CONVERT_POS
  -------         DO            
  X:000AH         SYMBOL        l
  -------         ENDDO         
  C:32CCH         LINE#         169
  C:32CCH         LINE#         170
  C:32CCH         LINE#         171
  C:32D1H         LINE#         172
  C:32EDH         LINE#         173
  C:32EDH         LINE#         174
  C:32F3H         LINE#         175
  C:335EH         LINE#         176
  C:33C9H         LINE#         177
  C:33C9H         LINE#         178
  C:33CEH         LINE#         179
  -------         ENDPROC       CONVERT_POS
  -------         PROC          TOUCH_ADJUST
  -------         DO            
  X:0006H         SYMBOL        vx1
  X:000AH         SYMBOL        vx2
  X:000EH         SYMBOL        vy1
  X:0012H         SYMBOL        vy2
  X:0016H         SYMBOL        chx1
  X:0018H         SYMBOL        chx2
  X:001AH         SYMBOL        chy1
  X:001CH         SYMBOL        chy2
  X:001EH         SYMBOL        lx
  X:0020H         SYMBOL        ly
  X:0022H         SYMBOL        p
  X:0042H         SYMBOL        cnt
  -------         ENDDO         
  C:1373H         LINE#         184
  C:1373H         LINE#         185
  C:1373H         LINE#         190
  C:1378H         LINE#         191
  C:1379H         LINE#         192
  C:1381H         LINE#         193
  C:1389H         LINE#         194
  C:138EH         LINE#         195
  C:1396H         LINE#         196
  C:1396H         LINE#         197
BL51 BANKED LINKER/LOCATER V6.22                                                      01/21/2022  11:42:17  PAGE 22


  C:1399H         LINE#         198
  C:1399H         LINE#         199
  C:1399H         LINE#         200
  C:139CH         LINE#         201
  C:139CH         LINE#         202
  C:13A2H         LINE#         203
  C:13A2H         LINE#         204
  C:13C2H         LINE#         205
  C:13DEH         LINE#         206
  C:13E4H         LINE#         207
  C:13E4H         LINE#         208
  C:13F6H         LINE#         209
  C:13F6H         LINE#         210
  C:13F6H         LINE#         211
  C:13FDH         LINE#         212
  C:1400H         LINE#         213
  C:1400H         LINE#         214
  C:1400H         LINE#         215
  C:1402H         LINE#         216
  C:1404H         LINE#         217
  C:1404H         LINE#         218
  C:140BH         LINE#         219
  C:140EH         LINE#         220
  C:140EH         LINE#         221
  C:140EH         LINE#         222
  C:1410H         LINE#         223
  C:1413H         LINE#         224
  C:1413H         LINE#         225
  C:141AH         LINE#         226
  C:141DH         LINE#         227
  C:141DH         LINE#         228
  C:141DH         LINE#         229
  C:1425H         LINE#         230
  C:1428H         LINE#         231
  C:1428H         LINE#         232
  C:142FH         LINE#         233
  C:1432H         LINE#         234
  C:1432H         LINE#         235
  C:1432H         LINE#         236
  C:14DDH         LINE#         237
  C:1585H         LINE#         238
  C:1618H         LINE#         239
  C:16C0H         LINE#         241
  C:176BH         LINE#         242
  C:1813H         LINE#         243
  C:18A6H         LINE#         244
  C:194EH         LINE#         247
  C:1A8CH         LINE#         248
  C:1A8CH         LINE#         249
  C:1A91H         LINE#         250
  C:1A98H         LINE#         251
  C:1AA3H         LINE#         252
  C:1AA6H         LINE#         253
  C:1AA6H         LINE#         254
  C:1B0CH         LINE#         255
  C:1B4EH         LINE#         258
  C:1B55H         LINE#         259
BL51 BANKED LINKER/LOCATER V6.22                                                      01/21/2022  11:42:17  PAGE 23


  C:1B5CH         LINE#         260
  C:1B64H         LINE#         262
  C:1B71H         LINE#         263
  C:1BBEH         LINE#         264
  C:1BD3H         LINE#         265
  C:1C22H         LINE#         266
  C:1C37H         LINE#         267
  C:1C80H         LINE#         268
  C:1C95H         LINE#         269
  C:1CDEH         LINE#         271
  C:1CEEH         LINE#         272
  C:1D3CH         LINE#         273
  C:1D53H         LINE#         274
  C:1DA3H         LINE#         275
  C:1DBAH         LINE#         276
  C:1E04H         LINE#         277
  C:1E1BH         LINE#         278
  C:1E65H         LINE#         280
  C:1E75H         LINE#         281
  C:1EBDH         LINE#         282
  C:1ED4H         LINE#         283
  C:1F1EH         LINE#         284
  C:1F35H         LINE#         285
  C:1F7FH         LINE#         286
  C:1F96H         LINE#         287
  C:1FE0H         LINE#         289
  C:1FF7H         LINE#         290
  C:2009H         LINE#         291
  C:200CH         LINE#         293
  C:2013H         LINE#         295
  C:2013H         LINE#         296
  C:2013H         LINE#         297
  C:2013H         LINE#         298
  -------         ENDPROC       TOUCH_ADJUST
  -------         PROC          POINT
  -------         DO            
  X:0006H         SYMBOL        t
  -------         ENDDO         
  C:3598H         LINE#         299
  C:3598H         LINE#         300
  C:3598H         LINE#         301
  C:35A2H         LINE#         303
  C:35A2H         LINE#         304
  C:35A2H         LINE#         305
  C:35A8H         LINE#         306
  C:35A8H         LINE#         307
  C:35B2H         LINE#         308
  C:35B8H         LINE#         309
  C:35B8H         LINE#         312
  C:35EBH         LINE#         313
  C:361EH         LINE#         314
  C:362FH         LINE#         315
  C:362FH         LINE#         317
  C:3632H         LINE#         319
  C:3632H         LINE#         320
  C:3650H         LINE#         321
  C:3670H         LINE#         322
BL51 BANKED LINKER/LOCATER V6.22                                                      01/21/2022  11:42:17  PAGE 24


  -------         ENDPROC       POINT
  -------         ENDMOD        TOUCH

  -------         MODULE        ?C?FPADD
  C:201BH         PUBLIC        ?C?FPADD
  C:2017H         PUBLIC        ?C?FPSUB
  -------         ENDMOD        ?C?FPADD

  -------         MODULE        ?C?FPMUL
  C:210CH         PUBLIC        ?C?FPMUL
  -------         ENDMOD        ?C?FPMUL

  -------         MODULE        ?C?FPDIV
  C:2215H         PUBLIC        ?C?FPDIV
  -------         ENDMOD        ?C?FPDIV

  -------         MODULE        ?C?FPCMP
  C:22B4H         PUBLIC        ?C?FPCMP
  C:22B2H         PUBLIC        ?C?FPCMP3
  -------         ENDMOD        ?C?FPCMP

  -------         MODULE        ?C?FCAST
  C:2335H         PUBLIC        ?C?FCASTC
  C:2330H         PUBLIC        ?C?FCASTI
  C:232BH         PUBLIC        ?C?FCASTL
  -------         ENDMOD        ?C?FCAST

  -------         MODULE        ?C?CASTF
  C:2369H         PUBLIC        ?C?CASTF
  -------         ENDMOD        ?C?CASTF

  -------         MODULE        ?C?CLDPTR
  C:23EAH         PUBLIC        ?C?CLDPTR
  -------         ENDMOD        ?C?CLDPTR

  -------         MODULE        ?C?IMUL
  C:2403H         PUBLIC        ?C?IMUL
  -------         ENDMOD        ?C?IMUL

  -------         MODULE        ?C?UIDIV
  C:2415H         PUBLIC        ?C?UIDIV
  -------         ENDMOD        ?C?UIDIV

  -------         MODULE        ?C?IILDX
  C:246AH         PUBLIC        ?C?IILDX
  -------         ENDMOD        ?C?IILDX

  -------         MODULE        ?C?ISTPTR
  C:2480H         PUBLIC        ?C?ISTPTR
  -------         ENDMOD        ?C?ISTPTR

  -------         MODULE        ?C?LMUL
  C:249FH         PUBLIC        ?C?LMUL
  -------         ENDMOD        ?C?LMUL

  -------         MODULE        ?C?ULDIV
  C:252AH         PUBLIC        ?C?ULDIV
BL51 BANKED LINKER/LOCATER V6.22                                                      01/21/2022  11:42:17  PAGE 25


  -------         ENDMOD        ?C?ULDIV

  -------         MODULE        ?C?LNEG
  C:25BCH         PUBLIC        ?C?LNEG
  -------         ENDMOD        ?C?LNEG

  -------         MODULE        ?C?ULCMP
  C:25CAH         PUBLIC        ?C?ULCMP
  -------         ENDMOD        ?C?ULCMP

  -------         MODULE        ?C?LSTXDATA
  C:25DBH         PUBLIC        ?C?LSTXDATA
  -------         ENDMOD        ?C?LSTXDATA

  -------         MODULE        ?C?LSTKXDATA
  C:25E7H         PUBLIC        ?C?LSTKXDATA
  -------         ENDMOD        ?C?LSTKXDATA

Program Size: data=9.0 xdata=169 code=16047
LINK/LOCATE RUN COMPLETE.  0 WARNING(S),  0 ERROR(S)
